:100000001CC035C034C033C032C031C030C02FC076
:100010002EC0E4C12CC02BC02AC029C028C027C0D4
:1000200026C05EC024C092C0A0C0ABC0B9C0C7C0CB
:10003000E3C0EDC0F6C003C107C111241FBECFE568
:10004000D4E0DEBFCDBF10E0A0E6B0E0EAE8F4E027
:1000500002C005900D92AA38B107D9F711E0AAE8BD
:10006000B0E001C01D92AE30B107E1F701C0C8CFCA
:10007000CFE5D4E0DEBFCDBFE6D1BC9A86E990E003
:1000800007D1882311F4C49AFFCF789440E050E060
:100090004431510589F0453151053CF44115510574
:1000A00059F04A30510551F00DC04E31510531F033
:1000B0004436510529F006C0C49A04C0C49802C051
:1000C0004FEF5FEF4F5F5F4F20918A0030918B00C1
:1000D00080918A0090918B0082179307C9F3D8CF43
:1000E0001F920F920FB60F9211242F933F934F93AD
:1000F0005F936F937F938F939F93AF93BF93EF9390
:10010000FF93BDD086B7806886BFFF91EF91BF9106
:10011000AF919F918F917F916F915F914F913F919F
:100120002F910F900FBE0F901F901895CF93DF93D4
:10013000EC018A819927AA27BB27FC013197EA3075
:10014000F10508F091C0ED5EFF4F0994FE01339672
:1001500082E08B8381E0818384EC93E093838283CC
:1001600084E08A8385E090E081C0EC81E83008F08B
:10017000E0E081E08A83FF27EE0FFF1FE05AFF4F88
:100180001AC0FE0134968C8131812281883008F0BA
:1001900080E0E82FFF27EE0FFF1FE458FF4F1DC040
:1001A000EC81E83008F0E0E081E08A83FF27EE0F81
:1001B000FF1FE259FF4F0190F081E02D2DC0FE019D
:1001C00034968C8131812281883008F080E0E82FDC
:1001D000FF27EE0FFF1FE259FF4FA081B181932F40
:1001E00090958C9189238C930190F081E02D2323AD
:1001F0008081822B808335C08C8187B9369A36996D
:10020000FECF82E08A8384B18B8385B114C08C8158
:10021000E82FFF2781E08A8380818B8382E090E052
:1002200025C08C81E82FFF272081318182E08A83DD
:100230002B83832F99278C8383E090E017C08C81D8
:10024000E82FFF278D81D6CFFE0134968C81A82F11
:10025000BB2782819381892F99272281FD01818388
:100260002C9380E090E002C0CE0166D0DF91CF9168
:100270000895E0918D00F0918E0009950895E09128
:100280008F00F091900088ED90E0099599270895EE
:10029000CF93DF93EC0122E038E1F901859194914D
:1002A0008750904B61F424E038E1F90125913491B5
:1002B000220F331FF90185919491039718F480E080
:1002C00090E037C02E5F3F4F46E050E0B9018DE827
:1002D00090E0D2D092B186E3E8EDF0E0282F1192C1
:1002E0002A95E9F78093D80081E08093D900809324
:1002F000DA001092DC001092DB00D093DE00C09395
:10030000DD0084B38F7C84BB85B38F7C85BB80E2AA
:1003100080B986B7846086BF86B7806886BF86B797
:10032000816086BF86B7806486BF9E7F92B981E078
:1003300090E0DF91CF910895E0919100F0919200CB
:10034000BC0183E990E009950895009731F0A2E09F
:10035000B0E01197F1F70197D1F70895009731F0C8
:10036000A0EDB7E01197F1F70197D1F70895CF937A
:10037000C82F882329F084E690E0E7DFC150D9F741
:10038000CF910895CF93C82F882329F08AE090E079
:10039000DCDFC150D9F7CF910895CF93C82F8823C0
:1003A00029F084E690E0DADFC150D9F7CF910895C3
:1003B000CF93C82F882329F08AE090E0CFDFC15087
:1003C000D9F7CF910895CF93C82F882329F081E0E2
:1003D00090E0C4DFC150D9F7CF9108951F920F92DA
:1003E0000FB60F9211248F939F9380918C008F5F93
:1003F00080938C008A3058F010928C0080918A0093
:1004000090918B00019690938B0080938A0083E8F3
:1004100082BF9F918F910F900FBE0F901F901895E4
:1004200083E083BF12BE81E089BF78940895209154
:100430008A0030918B0080918A0090918B00821706
:100440009307C9F308958FEF88BB17BA85BB14BA19
:1004500082BB11BA12BC10BC8CE089B91BB888E908
:100460008AB98EE080BD87EC86B986B1877C11F0B1
:100470003699FECFD5DF0895FB01DC0102C005905F
:0A0480000D9241505040D8F7089546
:10048A0036003600330030003600360036003700BA
:10049A0037003400310037003700370038003800A1
:0A04AA003500320038003800380039
:00000001FF
